:020000040000FA
:0400000094EF0DF07C
:08000800056ED8CF06F0E0CF31
:1000100007F00001E9CF0DF0EACF08F0E1CF09F0D9
:10002000E2CF0AF0D9CF0BF0DACF0CF0F3CF14F017
:10003000F4CF15F0FACF16F000C00FF001C010F0A9
:1000400002C011F003C012F004C013F0A0AA2CEFFC
:1000500000F0A1BA24EF08F00FC000F010C001F0CA
:1000600011C002F012C003F013C004F00DC0E9FF8C
:1000700008C0EAFF088E09C0E1FF0AC0E2FF0BC01A
:10008000D9FF0CC0DAFF14C0F3FF15C0F4FF16C08F
:10009000FAFF055007C0E0FF06C0D8FF1000F76A5E
:1000A000AE0FF66E000EF7220900F55012000403A1
:1000B000000000000000000000000000000008AE8A
:1000C00003D0F2CF0EF0F29EF76AE00FF66E000E4C
:1000D000F7220900F55008AE02D00EBEF28E1200D3
:1000E00040000800000000000000000000000000C8
:1000F0000000000000000000000000000000000000
:10010000F76A100FF66E010EF7220900F550120083
:100110000600FF0901A101190129081580257F7535
:10012000089508810819012908750895089108C0E3
:10013000F76A400FF66E010EF7220900F550120023
:100140000000F76A520FF66E010EF7220900F55013
:1001500012002000F76A640FF66E010EF722090004
:10016000F550120009022900010100C03209040003
:100170000002030000000921000100012220000705
:100180000581030800010705010308000100F76A63
:100190009E0FF66E010EF7220900F55012000100C5
:1001A000F76AB00FF66E010EF7220900F550120043
:1001B000120110010000004061044610000101021C
:1001C0000001F76AD20FF66E010EF7220900F55012
:1001D00012000403090408035400440045002C03E2
:1001E0005400650063006800440065007300690006
:1001F00067006E0020004D006F00640075006C0009
:1002000065002000300034003600F2CF0EF0F29E80
:10021000F76A240FF66E020EF7220900F5500EBEA3
:10022000F28E120020636F6E6669673D25782000AC
:10023000F2CF0EF0F29EF76A4A0FF66E020EF72228
:100240000900F5500EBEF28E120020737461743DE9
:1002500025782000F2CF0EF0F29EF76A6E0FF66E50
:10026000020EF7220900F5500EBEF28E1200205346
:100270005155414C5F6D6F7573653D2578200000C9
:10028000F2CF0EF0F29EF76A9A0FF66E020EF72288
:100290000900F5500EBEF28E1200206D61785F707D
:1002A0006978656C3D2564200000F2CF0EF0F29E67
:1002B000F76AC40FF66E020EF7220900F5500EBE63
:1002C000F28E1200206D696E5F706978656C3D2555
:1002D00064200000F2CF0EF0F29EF76AEE0FF66E89
:1002E000020EF7220900F5500EBEF28E1200206CAD
:1002F00064725F696E5F613D254C64200A0D0000E9
:10030000F2CF0EF0F29EF76A1A0FF66E030EF72286
:100310000900F5500EBEF28E1200207368757474D9
:1003200065725F75707065723D2564200000F2CFC4
:100330000EF0F29EF76A480FF66E030EF7220900E0
:10034000F5500EBEF28E12002073687574746572DB
:100350005F6C6F7765723D2564200000F2CF0EF070
:10036000F29EF76A760FF66E030EF7220900F5503B
:100370000EBEF28E1200206672616D655F7065724E
:10038000696F643D25642000F2CF0EF0F29EF76A9B
:10039000A20FF66E030EF7220900F5500EBEF28E84
:1003A00012000A0A0D20303436202D204D6F75734F
:1003B00065204D6F64756C65200A0A0D0000F2CF50
:1003C0000EF0F29EF76AD80FF66E030EF7220900C0
:1003D000F5500EBEF28E12000D0A2D2D3E205265F4
:1003E00063656976656420646174613A20307825BC
:1003F0005820307825580A0D0000F2CF0EF0F29EFA
:10040000F76A140FF66E040EF7220900F5500EBEBF
:10041000F28E12000D0A3C2D2D2053656E64696E1C
:10042000672062797465733A2030782558203078D7
:100430002558203078255820307825580000F2CFF4
:100440000EF0F29EF76A580FF66E040EF7220900BE
:10045000F5500EBEF28E12000D0A0A55534220636B
:100460006F6E6E65637465642C2077616974696E64
:100470006720666F7220656E756D65726174696F55
:100480006E2E2E2E0000F2CF0EF0F29EF76AA00F15
:10049000F66E040EF7220900F5500EBEF28E120021
:1004A0000D0A0A55534220646973636F6E6E65636B
:1004B0007465642C2077616974696E6720666F7259
:1004C00020636F6E6E656374696F6E2E2E2E000052
:1004D000F2CF0EF0F29EF76AEA0FF66E040EF722E4
:1004E0000900F5500EBEF28E12000D0A0A55534255
:1004F00020656E756D657261746564206279205047
:10050000432F484F53540000F2CF0EF0F29EF76A8B
:10051000220FF66E050EF7220900F5500EBEF28E80
:1005200012000D0A0A55534220756E656E756D6591
:1005300072617465642062792050432F484F535490
:100540002C2077616974696E6720666F7220656E12
:10055000756D65726174696F6E2E2E2E00006D923E
:10056000699468942FEF08F06A6A689238EF08F08F
:100570000101EA6BEA530AE1036AEA512D0FE96EC1
:10058000000E0320EA6EEF6AEA2BF4D7206A010E10
:10059000216E1F6A0001000C010E0101F36FF3517F
:1005A0000F080EE3700EF325016E0F0E036ED8B028
:1005B000032A01C0E9FF03C0EAFFEF6AF32BEFD77C
:1005C000246A236A0001000C400E0401016F050E2D
:1005D000036F026B880E006F046B050E076F400EF1
:1005E000066F0001000C6A6A686A9F0E6B6E390E16
:1005F000696E6E6ABDDFD0DF160E706E68A602D01F
:100600006896FCD76D98E0DF030E256E3EEF08F08C
:10061000698468986D8244EF08F0689C4AEF08F09E
:1006200070A002D0D1DF7090689A50EF08F0EEC150
:1006300026F0000CFF0E266E000C0101EC6B2C5214
:1006400044E0EC513F0841E32250FC0F31E2040F3B
:10065000000170EF03F0036A2B50F2CFEEF1F29E2F
:1006600079DD0101EEBFF28EED6F22D0036A2B50CF
:10067000F2CFEEF1F29E44DD0101EEBFF28EED6F9E
:1006800017D0036A2B50F2CFEEF1F29E9ADD0101F2
:10069000EEBFF28EED6F0CD0036A2B50F2CFEEF16D
:1006A000F29E7EDD0101EEBFF28EED6F01D0010101
:1006B0002B2A2C06EC51EC2B036A400FE96E050E39
:1006C0000320EA6EEDC1EFFFBAD72C5204E1EC51E2
:1006D000400801E01F6AECC1EEF10001A8DF000C48
:1006E000E824F76AF736FB0FF66E060EF7220A00CB
:1006F000F550FA6E0800F550F96E56066C06820643
:1007000098062B6A226A05010351010A000109E0DB
:10071000030A0CE0010A0DE0220A24E0030A36E095
:1007200061D0120E2C6E030E226E5ED0290E2C6E3E
:100730005BD0020E226E036A05010251270FE96E9B
:10074000000E0320EA6EEFCF2BF0036A2B50F2CF9E
:10075000ECF1F29E000135DD0101ECBFF28E2C6E52
:10076000000142D0120E2B6E2B3C01D00DD0036A3B
:100770002B50F2CFECF1F29EEDDC0101ECBFF28EDA
:100780002C6E000131D002D055DF3AD0D89005014F
:100790000435036AF2CFECF1F29E0001C9DC0900D6
:1007A000F5CF03F00101ECBFF28E2B6E2B3C01D094
:1007B00016D0010E226ED89005010435036AF2CFDF
:1007C000ECF1F29E0001BDDC0900F5CF03F0010160
:1007D000ECBFF28E2C6E000107D004D001010001A5
:1007E00029DF0ED027DF0CD00501075305E12C507F
:1007F000065D02E206C52CF0010E1F6E00011DDF32
:10080000000C0101EB5306E1040E256E0001C4DE6D
:10081000D1D00101050E256EEE6F800EED6F010E39
:10082000EC6FEC510F08D8A0C5D0EF6B036AEC5108
:10083000F2CFF3F1F29E000132DC0101F3BFF28E40
:10084000000A55E0040EEF6FD890EC35036AF2CF42
:10085000F3F1F29E000133DC0900F5CF03F0010152
:10086000F3BFF28EF06F03C0F1F1EC51080DF350BD
:10087000010F016E040E036ED8B0032A01C0E9FF18
:1008800003C0EAFFF0C1EFFFEC51080DF350020F77
:10089000016E040E036ED8B0032A01C0E9FF03C045
:1008A000EAFFEEC1ECFFED52EDC1EFFFD890EC3561
:1008B000036AF2CFF3F1F29E000101DC0900F5CFEB
:1008C00003F00101F3BFF28EED270350EE23880EF3
:1008D000F26FF1B1F281F1B3F283EC51080DF3CF75
:1008E00001F0040E01C0E9FFEA6EF2C1EFFF036AF6
:1008F000EC51F2CFF3F1F29E00014FEC00F0010158
:10090000F3BFF28E000A34E0EF83EC51080DF35090
:10091000060F016E040E036ED8B0032A01C0E9FF72
:1009200003C0EAFFEEC1ECFFED52EDC1EFFFD8903E
:10093000EC35036AF2CFF3F1F29E00015FEC00F0B8
:100940000900F5CF03F00101F3BFF28EED2703504C
:10095000EE23EC51080DF350040F016E040E036EEC
:10096000D8B0032A01C0E9FF03C0EAFF400EEF6ED2
:10097000EF51060802E10E0EEF6F036AEC51F2CF61
:10098000F3F1F29E00014FEC00F00101F3BFF28E93
:10099000020801E0EF89700EEC25016E0F0E036E68
:1009A000D8B0032A01C0E9FF03C0EAFFEFC1EFFF9F
:1009B000EC2B37D700012EEF05F0050101510001A6
:1009C0000DE0010A15E0020A20E0060A2AE0030A07
:1009D00031E00E0A31E0010A37E046D021C040F58F
:1009E0000501416B020E0101EE6F000120DE3ED0D9
:1009F0000501022D07D0010E21160101EE6B000149
:100A000016DE02D0000116DE31D00501022D06D01F
:100A100021820101EE6B00010ADE02D000010ADE34
:100A200025D0020E1F6E02C52AF00101EE6B0001F7
:100A3000FEDD1CD066DE1AD020C040F5010E01019B
:100A4000EE6F0001F4DD12D00501025101080AE346
:100A500002C520F002C5EBF10001D3D60101EE6B17
:100A60000001E5DD000102D0E5DD00D083EF06F0F6
:100A700020C0EBF105010151000107E00A0A0EE078
:100A8000010A34E00D0A47E048D00501406B416B94
:100A9000020E0101EE6F0001CADD41D00101EB53EE
:100AA00022E0010EEB5D036AF2CFEDF1F29E000150
:100AB000C7EC00F00101EDBFF28E016E0501045D8F
:100AC000D8A002D001010FD0036A04512D0FE96EA6
:100AD000000E0320EA6EEFCF40F5010E0101EE6F2C
:100AE0000001A5DD02D00001A5DD19D00101EB5305
:100AF0000FE0036A050104512D0FE96E000E03207B
:100B0000EA6E02C5EFFF0101EE6B000190DD02D03D
:100B1000000190DD04D0F5DD02D08CDD00D083EF44
:100B200006F00101EC91EBBFEC81EB9FECA113D03F
:100B3000036AEB51F2CFEDF1F29E00014FEC00F0B1
:100B40000101EDBFF28E000A02E1000E01D0010E9C
:100B5000016E13D012D0036AEB51F2CFEDF1F29E89
:100B600000014FEC00F00101EDBFF28E000A02E13E
:100B7000000E01D0010E016E00D0000136EF06F02C
:100B80000101EC91EBBFEC81EB9FECA110D0EB519C
:100B9000080DF350040F016E040E036ED8B0032A43
:100BA00001C0E9FF03C0EAFF880EEF6E09D0EB51E8
:100BB000080DF3CF01F0040E01C0E9FFEA6EEF6A01
:100BC000000145EF06F00101EC91EBBFEC81EB9FDA
:100BD000ECA110D0EB51080DF350040F016E040E80
:100BE000036ED8B0032A01C0E9FF03C0EAFF840EF8
:100BF000EF6E0AD0EB51080DF3CF01F0040E01C0E7
:100C0000E9FFEA6E840EEF6E00014DEF06F0010180
:100C1000EC91EBBFEC81EB9FECA110D0EB51080DF8
:100C2000F350040F016E040E036ED8B0032A01C006
:100C3000E9FF03C0EAFFEFCFEDF10AD0EB51080D59
:100C4000F3CF01F0040E01C0E9FFEA6EEFCFEDF142
:100C5000EDAF02D0EDB502D0000E01D0010E016E55
:100C6000000159EF06F004C5EBF15BD701522EE00D
:100C700005010151010A000105E0020A0BE0030A27
:100C800011E022D004C5EBF17BD70101EE6B00012E
:100C9000CEDC1CD004C5EBF196D70101EE6B000150
:100CA000C6DC14D00501406B416B04C5EBF10001BB
:100CB000AED7015203E0010E0501406F020E0101A3
:100CC000EE6F0001B4DC02D0B5DC00D083EF06F09B
:100CD0000501015100D00001ADDC00D083EF06F02A
:100CE0001F6A050100517F0B000107E0010A06E0C1
:100CF000030A05E0230A04E004D05FD6B9D6B3D7CF
:100D0000E7D798DC00D0BDEF07F00101EB51080DEB
:100D1000F3CF01F0040E01C0E9FFEA6EEFCFEDF171
:100D2000EC51020806E1EDAD02D0EC6B02D0010EF1
:100D3000EC6FEC51030812E1840EED6FEB51080DDE
:100D4000F350040F016E040E036ED8B0032A01C0E5
:100D5000E9FF03C0EAFF840EEF6E09D0EC2D03D04B
:100D6000C80EED6F04D0EC5302E1880EED6F036AFC
:100D7000010E026EEB51006E05E0D890023603368C
:100D8000002EFBD70250FF0A006EFF0E031A005020
:100D9000231603502416D890EB35036AF2CFF0F1F6
:100DA000F29E00015FEC00F00900F5CF03F00101B5
:100DB000F0BFF28EEE6F03C0EFF1EB51080DF35070
:100DC000010F016E040E036ED8B0032A01C0E9FFC3
:100DD00003C0EAFFEEC1EFFFEFB1ED81EFB3ED83AA
:100DE000EB51080DF3CF01F0040E01C0E9FFEA6EEC
:100DF000EDC1EFFF0001000C0101EB51080DF350B4
:100E0000040F016E040E036ED8B0032A01C0E9FF7F
:100E100003C0EAFFEFCFEFF1EFBF5BD0EB51080D5E
:100E2000F350050F016E040E036ED8B0032A01C003
:100E3000E9FF03C0EAFFECC1EFFFEE51020816E143
:100E4000EB51080DF350040F016E040E036ED8B081
:100E5000032A01C0E9FF03C0EAFFEFCFEFF1EFADD6
:100E600002D0EE6B02D0010EEE6F13D0EE510408EB
:100E700010E1EB51080DF3CF01F0040E01C0E9FFC2
:100E8000EA6EEFCFEFF1EFAD03D0010EEE6F01D0C0
:100E9000EE6BEE2D03D0C80EEF6F04D0EE5302E1DF
:100EA000880EEF6FEDB1EF81EDB3EF83EB51080DDD
:100EB000F350040F016E040E036ED8B0032A01C074
:100EC000E9FF03C0EAFFEFC1EFFF010E016E03D09F
:100ED00000D0000E016E0001000C0101EB5305E192
:100EE0000001E4EC02F010D00101036A010E026E71
:100EF000EB51006E05E0D89002360336002EFBD78A
:100F000002502312035024120001000CECC16EFFAA
:100F10000101EC5303E0040E256E02D0020E256E93
:100F2000000198EF07F0206A1F6A2AC0ECF1EED7A3
:100F3000A9EF07F00101EB530DE11F2C05D00001D3
:100F40001DEC03F006D001011F50020803E100016F
:100F5000EAD701010001000C6C300101EA6FEA33AD
:100F6000EA331F0EEA176C5246E1040100513C0BB4
:100F7000340821E1046B0001B3D6263C07D00101FF
:100F8000EB6B030EEC6F0001C0DE12D00101EB6BC6
:100F9000020EEC6F0001B9DE2650FE0809E00101E7
:100FA000EB6BED6B26C0ECF1040EEE6F000124DF5D
:100FB0006D981ED0040100513C0B04081AE1010198
:100FC000EB6B00018ADF0101EB6B020EEC6F00019D
:100FD0009CDE2650FE080CE0263C01D009D0010121
:100FE000EB6BED6B26C0ECF1010EEE6F000104DF40
:100FF000040127D001016C50040816E1FF0E266E93
:10100000EB6B000197DF263C01D00AD00101EB6BAE
:10101000ED6B26C0ECF1020EEE6F0001EDDE02D0AA
:10102000E4EC02F00DD001016CB406D0EAC1EBF1A2
:10103000000153DF05D00101EAC1EBF100017ADFC5
:101040000401000155EF08F0255201E12FD068524C
:101050002DE068A404D069A402D0AFEF02F06DA225
:1010600001D024D068A204D069A202D0B4EF02F06B
:1010700068A004D069A002D0F3EF02F068A804D001
:1010800069A802D008EF03F068AC04D069AC02D0C4
:101090000DEF03F068AA04D069AA02D010EF03F0A4
:1010A00068A604D069A602D057D76896A19A2CEFFB
:1010B00000F06D6A696A080E6F6E94503009010184
:1010C000946E256A186AF2BE188EF29E0001B8EC82
:1010D00002F018BEF28E246A236A92EF08F0186AB2
:1010E000F2BE188EF29EB8EC02F018BEF28E6D6A57
:1010F000140E6F6E696A6D86010E256E83EF08F01F
:101100006DB601D0ECD7252C0BD06DBA09D0686A2A
:10111000696AA08AC00EF212110E696E020E256E67
:10112000000CC7D7EDDF25500208FCE1CBEF0DF036
:101130009EA8FED7AD6E000C030E0101E25F0BE32B
:10114000010EEA6EE20EE96EEF5005E002D000D02B
:101150000000EF2EFCD70001E2EF08F00101E06B88
:10116000E16B040E936E8182DC2D04D0DD51800989
:10117000E06F04D0DC5302E1DDC1E0F1070EDF6F68
:10118000DF3D01D01BD08192060E006E002EFED7EF
:101190000000E0C100F0DF51016E04E0D8900032A1
:1011A000012EFCD700A0819000B081808182060EC4
:1011B000006E002EFED70000DF07E2D7C80EE26FF8
:1011C0000001BAD70101DC5302E1050E936E070E50
:1011D000DF6FDF3D01D02DD08192060E006E002E14
:1011E000FED70000DC530EE181A00BD0010E006E93
:1011F000DF51016E04E0D8900036012EFCD700507C
:10120000E1130FD0DC2D0DD0DEC100F0DF51016EF7
:1012100004E0D8900032012EFCD700A0819000B0ED
:1012200081808182060E006E002EFED70000DF074F
:10123000D0D7040E936EE1C101F00001000C010E45
:10124000EA6ED80EE96EEF500EE0070E016E006AEE
:10125000002EFED7012EFBD7C70E006E002EFED744
:101260000000EF2EF2D7000C010E0101D86F20C054
:10127000D9F1D8530FE0D4530DE1DA6BDA51000104
:101280001FEC02F00101DA2B000152DF2C0E0101EC
:10129000DA5DF4E1D8530FE1D4530DE0DA6BDA51A3
:1012A000000143EC02F00101DA2B000141DF2E0EB8
:1012B0000101DA5DF4E1D9530FE0D5530DE1DA6BAA
:1012C000DA51000168EC02F00101DA2B000130DF95
:1012D0001C0E0101DA5DF4E1D9530FE1D5530DE0A5
:1012E000DA6BDA51000184EC02F00101DA2B000123
:1012F0001FDF3A0E0101DA5DF4E1D8C1D4F1D9C1A2
:10130000D5F10001000C0101DD51080DF350020F71
:10131000016E040E036ED8B0032A01C0E9FF03C0BA
:10132000EAFFECCF03F0ED52EFCFE2F103C0E3F1BF
:10133000DD51080DF350010F016E040E036ED8B09D
:10134000032A01C0E9FF03C0EAFFEF50036AE56F1B
:1013500003C0E6F1DD51080DF3CF01F0040E01C02A
:10136000E9FFEA6EEFCFE4F1E4B1E681E4B3E683AE
:10137000E651E15D08E303E1E051E55D04E2E6C129
:10138000E1F1E5C1E0F1E66BE56BE651E15D1AE301
:1013900003E1E051E55D16E2E2C1E9FFE3C1EAFFE6
:1013A000EFCFE9F1DFC1EAFFDEC1E9FFE9C1EFFFFD
:1013B000DE2BD8B4DF2BE22BD8B4E32BE52BD8B44B
:1013C000E62BE3D7E0C101F0E1C102F00001F4EF48
:1013D00009F0D8C1DDF1DAC1DFF1D9C1DEF1DCC13C
:1013E000E1F1DBC1E0F18FD702C0DCF101C0DBF13C
:1013F000186AF2BE188EF29ED8C1EBF1020E0101FE
:10140000EC6F000182DC18BEF28E0101DBC101F03D
:10141000DCC102F00001000C0101DEBF10D00F0E94
:10142000006EDD3900160A0E005C03E2300E002665
:1014300002D0DE51002600509EA8FED7AD6E0F0EE2
:10144000DD170A0EDD5D02E2300E02D0DE9FDE51B6
:10145000DD27DD519EA8FED7AD6E0001000C010115
:10146000E451016AE35D03E2E3C100F00CD0006ADD
:10147000080EE56FE3370036E451005CD8B0006E2B
:101480000136E52FF7D70001000C200E0101DEA97F
:10149000300EDF6FDDC100F0DDAF07D0001E002A87
:1014A00000C0DDF12D0EDF6FDE8F0150DDC1E3F1F5
:1014B000640EE46F0001D3DF00C0DDF1300E0124C3
:1014C0000101E06FDDC1E3F10A0EE46F0001C7DF47
:1014D000300E00240101E26F300E0124E16FDFC104
:1014E00000F0DEA702D0DEAFDE95DEB90BD0DEAFB6
:1014F00022D0DEB520D000C0E0F1DEB31CD000C0A9
:10150000E1F119D0300EE05D16E100C0E0F1200EEF
:10151000DF6FDEA704D0DE95DE83DEAFDE93300E14
:10152000E15D09E100C0E1F1200EE06FDEA7F7D731
:10153000DE93DEAFDE91DEA504D0DF519EA8FED79C
:10154000AD6EDEA304D0E0519EA8FED7AD6EDEA145
:1015500004D0E1519EA8FED7AD6EE2519EA8FED701
:10156000AD6E0001000CEACFE5F1E9CFE4F1010135
:10157000DEAF08D0E48FE4A9E42BDD1FDE1FDD2BF6
:10158000D8B4DE2BDE39F009E06FE027E20FE16F1F
:10159000320FE36FDE510F0BE127E127E327E90F5D
:1015A000E26FE227E227DD390F0BE227E327E2377C
:1015B000E337E31FE337DD510F0BE327E037070E77
:1015C000DF6F0A0EE207E327FDE3E107E227FDE311
:1015D000E007E127FDE3DF07E027FDE3010EEA6E08
:1015E000DF0EE96E070EE415E49DE906E41507E158
:1015F000E4B9E92AE4B903D0200E006E1CD0E92634
:10160000E30EE95CD8B4E48DEF50006E08E1E4BD70
:1016100006D0E4B914D0E4B702D0200E0BD0E4AF6A
:1016200006D02D0E006EED50E49DE49F04D0E487BB
:10163000E499300E002600509EA8FED7AD6EEE5005
:10164000E4ADDED7000146EF0CF0746B0101D85118
:101650000001835D0EE0010E0101DC6F400EDD6FC5
:10166000800EDE6F00017ADDC70E006E002EFED701
:1016700000D0D8C183F00101D8510308D8B40ED1ED
:10168000D8510B08D8A00AD1DC6B400EDD6FDE6BA1
:10169000000164DD01C084F06751020816E1010118
:1016A000DC6BDC51000105EC01F00101DC2B0001D9
:1016B0003FDD080E0101DC5DF4E184C0DDF1570E71
:1016C000DE6F0001A9DE200E33DD0101DC6B410E6F
:1016D000DD6FDE6B000142DD01C085F0675102085D
:1016E00016E10101DC6BDC51000118EC01F0010195
:1016F000DC2B00011DDD060E0101DC5DF4E185C07F
:10170000DDF1570EDE6F000187DE200E11DD0101D5
:10171000DC6B420EDD6FDE6B000120DD01C086F068
:10172000675102080FE1200E03DD790E01DD3D0E49
:10173000FFDC86C0DDF11F0E0101DE6F0001A5DEBA
:10174000200EF6DC0101DC6B430EDD6FDE6B000169
:1017500005DD01C087F0675102080FE1200EE8DCCB
:10176000780EE6DC3D0EE4DC87C0DDF11F0E0101E2
:10177000DE6F00018ADE200EDBDC0101DC6B440E33
:10178000DD6FDE6B0001EADC01C088F06751020802
:1017900016E10101DC6BDC5100012AEC01F00101D2
:1017A000DC2B0001C5DC0D0E0101DC5DF4E188C01D
:1017B000DDF1570EDE6F00012FDE200EB9DC0101D6
:1017C000DC6B450EDD6FDE6B0001C8DC01C089F00B
:1017D0006751020816E10101DC6BDC51000140ECAD
:1017E00001F00101DC2B0001A3DC0B0E0101DC5D2B
:1017F000F4E189C0DDF11F0EDE6F000146DE200E30
:1018000097DC0101DC6B460EDD6FDE6B0001A6DCB0
:1018100001C08AF06751020816E10101DC6BDC515E
:10182000000155EC01F00101DC2B000181DC0B0E05
:101830000101DC5DF4E18AC0DDF11F0EDE6F000105
:1018400024DE200E75DC0101DC6B470EDD6FDE6BE4
:10185000000184DC716B01C070F0675102081CE16B
:101860000101DC6BDC5100016AEC01F00101DC2BB1
:1018700000015EDC0A0E0101DC5DF4E1100EE96E90
:1018800071C0DEF170C0DDF100016DD6200E50DCBC
:101890000A0E4EDC0D0E4CDCE5D00101D8510308D8
:1018A000D8A46ED0010EDC6F400EDD6F010EDE6F2E
:1018B000000154DC010E0101DC6F480EDD6FDE6BB0
:1018C00000014CDC0101DB6BDA6B010ED96FD951E1
:1018D000450803E1DA2D01D036D0D92D11D0DA53E5
:1018E0000FE1DB51C00BC0080AE0DC6B480EDD6F76
:1018F000DE6B000133DC01C0DBF10101F2D717D050
:10190000DC6B480EDD6FDE6B000128DC01C0DBF113
:101910000101DB51400B40080AE0DC6B480EDD6F33
:10192000DE6B00011BDC01C0DBF1F2D701018B0E85
:10193000D925E96E000EDA21EA6EDBC1EFFFD92B63
:10194000D8B4DA2BC4D7DC6B450EDD6FDE6B00013B
:1019500005DC01C089F00101DC6B460EDD6FDE6B3A
:101960000001AEEC08F001C08AF0010E0101DC6F4D
:10197000400EDD6FDE6B0001AEEC08F073D00101AC
:10198000D8510B08D8B06FD0DC6B490EDD6FDE6B21
:101990000001AEEC08F001C0D1F16751020818E176
:1019A0000101DC6BDC51000180EC01F00101DC2B5A
:1019B000000198EC08F00F0E0101DC5DF3E1D1C1EC
:1019C000DDF11F0EDE6F000160DD200E98EC08F0E7
:1019D0000101DC6B4A0EDD6FDE6B0001AEEC08F03E
:1019E00001C0D2F16751020818E10101DC6BDC5142
:1019F000000197EC01F00101DC2B000198EC08F0EC
:101A00000F0E0101DC5DF3E1D2C1DDF11F0EDE6FCF
:101A100000013BDD200E98EC08F00101DC6B4B0E61
:101A2000DD6FDE6B0001AEEC08F001C0D3F1675151
:101A3000020818E10101DC6BDC510001AEEC01F0A1
:101A40000101DC2B000198EC08F00E0E0101DC5DB9
:101A5000F3E1D3C1DDF11F0EDE6F000116DD200EB4
:101A600098EC08F00101000145EF0EF00101D8519A
:101A7000080DF350040F016E040E036ED8B0032A54
:101A800001C0E9FF03C0EAFFEFCFE0F1E0BF48D0BB
:101A9000D851080DF350060F016E040E036ED8B036
:101AA000032A01C0E9FF03C0EAFFECCF03F0ED52C7
:101AB000EFCFE1F103C0E2F1DF6BDE6BDF51DC5D04
:101AC0001AE303E1DB51DE5D16E2D9C1E9FFDAC1B9
:101AD000EAFFEFCFE5F1E2C1EAFFE1C1E9FFE5C1CD
:101AE000EFFFE12BD8B4E22BD92BD8B4DA2BDE2BC5
:101AF000D8B4DF2BE3D7186AF2BE188EF29ED8C195
:101B0000EBF1DCC1EDF1DBC1ECF1DDC1EEF1000187
:101B1000FCEC06F018BEF28E015004D000D001019A
:101B2000000E016E0001000CF86AD09E088EFE0EB9
:101B3000006E040E016E020EE96E000EEA6EEE6A91
:101B4000002EFDD7012EFBD7EA6AE96AB8960C0E83
:101B5000AF6EA60EAC6E900EAB6EC150C00B0F09EF
:101B6000C16E070EB46E196A1A6A256A276A040ED6
:101B7000286E0C0E296E2C6A666B0101D46BD56B36
:101B8000C00EF2122F0E926E040E936E950E946E8E
:101B9000000191EF08F0929889980101D86BD85113
:101BA0000001C4EC01F00101D82B000198EC08F011
:101BB0001A0E0101D85DF3E1010EDC6F400EDD6FFE
:101BC000800EDE6F0001AEEC08F0C70E006E002E36
:101BD000FED700D0020E676F010E6927D8B06A2BBE
:101BE000D8B46B2BD8B46C2B010E0101D86F000157
:101BF0001FEC09F080EC08F034EC09F02052D8B466
:101C000055D223A253D2010E0101D86FDA6B520EC6
:101C1000D96FDC6B020EDB6F0001E9EC09F001010A
:101C2000D86BD8510001DFEC01F00101D82B000185
:101C300098EC08F0170E0101D85DF3E152C0DDF118
:101C4000370EDE6F00010CEC0AF0200E98EC08F065
:101C5000300E98EC08F0780E98EC08F053C0DDF1E7
:101C6000370E0101DE6F00010CEC0AF00A0E98EC51
:101C700008F00D0E98EC08F0525201E000D05352DB
:101C800001E000D053C0D8F1E0D48351030823E031
:101C900083510B0820E384C04AF085C04BF086C016
:101CA0004CF087C04DF088C04EF089C04FF08AC01C
:101CB00050F070C051F0010E0101D86FDA6B4A0E7E
:101CC000D96FDC6B080EDB6F020EDD6F0001CEDE1C
:101CD000015200E0EBD183510B081BE2D1C14AF065
:101CE000D2C14BF0D3C14CF04D6A4E6A4F6A506A74
:101CF000516A010E0101D86FDA6B4A0ED96FDC6BA5
:101D0000080EDB6F020EDD6F0001B0DE015200E055
:101D1000CDD183510308D8A4C9D10101D66BD651C6
:101D20001208D8B41DD1D76BD7510308D8B416D137
:101D3000D6C14AF0D7C14BF0D651120DF350010F66
:101D4000D86FD751060DF350D8258B0FE96EEA6A8C
:101D5000D8B0EA2AEFCF4CF0D651120DF350020F53
:101D6000D86FD751060DF350D8258B0FE96EEA6A6C
:101D7000D8B0EA2AEFCF4DF0D651120DF350030F31
:101D8000D86FD751060DF350D8258B0FE96EEA6A4C
:101D9000D8B0EA2AEFCF4EF0D651120DF350040F0F
:101DA000D86FD751060DF350D8258B0FE96EEA6A2C
:101DB000D8B0EA2AEFCF4FF0D651120DF350050FED
:101DC000D86FD751060DF350D8258B0FE96EEA6A0C
:101DD000D8B0EA2AEFCF50F0D651120DF350060FCB
:101DE000D86FD751060DF350D8258B0FE96EEA6AEC
:101DF000D8B0EA2AEFCF51F0010ED86FDA6B4A0E55
:101E0000D96FDC6B080EDB6F020EDD6F00012EDE7A
:101E10000101D86BD8510001FDEC01F00101D82B74
:101E2000000198EC08F0170E0101D85DF3E14AC0FB
:101E3000DDF1370EDE6F00010CEC0AF0200E98EC9D
:101E400008F0300E98EC08F0780E98EC08F04BC0D3
:101E5000DDF1370E0101DE6F00010CEC0AF0200EFF
:101E600098EC08F0300E98EC08F0780E98EC08F03A
:101E70004CC0DDF1370E0101DE6F00010CEC0AF001
:101E8000200E98EC08F0300E98EC08F0780E98ECE4
:101E900008F04DC0DDF1370E0101DE6F00010CECE2
:101EA0000AF0200E98EC08F0300E98EC08F0780E4E
:101EB00098EC08F04EC0DDF1370E0101DE6F000135
:101EC0000CEC0AF0200E98EC08F0300E98EC08F0BC
:101ED000780E98EC08F04FC0DDF1370E0101DE6F8F
:101EE00000010CEC0AF0200E98EC08F0300E98EC93
:101EF00008F0780E98EC08F050C0DDF1370E0101C3
:101F0000DE6F00010CEC0AF0200E98EC08F0300EA9
:101F100098EC08F0780E98EC08F051C0DDF1370E1F
:101F20000101DE6F00010CEC0AF0320E0101D86FE6
:101F300000011FEC09F080EC08F034EC09F0010E10
:101F40000101D86FDA6B520ED96FDC6B020EDB6FBA
:101F50000001E9EC09F00101D72BE6D6D62BDFD63C
:101F6000120E4A6E4B6A4C6A4D6A4E6A89C04FF037
:101F70008AC050F0516A010ED86FDA6B4A0ED96FE1
:101F8000DC6B080EDB6F020EDD6F00016FDD0152AE
:101F900000E00101D86BD8510001FDEC01F0010116
:101FA000D82B000198EC08F0170E0101D85DF3E181
:101FB0004AC0DDF1370EDE6F00010CEC0AF0200E96
:101FC00098EC08F0300E98EC08F0780E98EC08F0D9
:101FD0004BC0DDF1370E0101DE6F00010CEC0AF0A1
:101FE000200E98EC08F0300E98EC08F0780E98EC83
:101FF00008F04CC0DDF1370E0101DE6F00010CEC82
:102000000AF0200E98EC08F0300E98EC08F0780EEC
:1020100098EC08F04DC0DDF1370E0101DE6F0001D4
:102020000CEC0AF0200E98EC08F0300E98EC08F05A
:10203000780E98EC08F04EC0DDF1370E0101DE6F2E
:1020400000010CEC0AF0200E98EC08F0300E98EC31
:1020500008F0780E98EC08F04FC0DDF1370E010162
:10206000DE6F00010CEC0AF0200E98EC08F0300E48
:1020700098EC08F0780E98EC08F050C0DDF1370EBF
:102080000101DE6F00010CEC0AF0200E98EC08F064
:10209000300E98EC08F0780E98EC08F051C0DDF1A5
:1020A000370E0101DE6F00010CEC0AF095D503003C
:020000040030CA
:0E00000000051E1F008381000FC00FE00F409F
:00000001FF
